:020000040000FA
:1000000031284334613470346134633469346D347D
:100010006534743472347534A0346F342E346B34D8
:100020002E34203420342034203420342034203422
:10003000A0344334203473346334753472347434EC
:100040002034203420342034A034443465347334D4
:1000500063346134723463346134203420342034A6
:10006000A03483160230810000308600831286019E
:1000700000308B001F149F121F129F119F171F1318
:1000800083169F019F1783123921803076212830F3
:100090008521633085212930852120308521443018
:1000A00085212E3085214F3085216C30852174309B
:1000B000852165308521613085216E30852175303F
:1000C000852101302B21FF30AC009721FF30AC009F
:1000D0009721FF30AC009721FF30AC009721FF3013
:1000E000AC009721FF30AC009721FF30AC00972186
:1000F000FF30AC00972139217D2893203008A300E0
:100100003108A400E82009210D302B21FF30AC007C
:100110009721FF30AC009721FF30AC009721FF30D2
:10012000AC0097217D28B32019302B21B001B101FB
:100130008030831681008312071483160710831200
:100140000714273081000B11C620A418AF28B00A6D
:100150000319B10A0319AF280B1DAC28A128831677
:1001600007148312080025302B210710831607106F
:1001700083120710C6202408031DBA28F83023056F
:10018000031DBA2883160714831208001F151F19B0
:10019000C7281E08A40083161E088312A3000800A7
:1001A0002108A30722080318220FA407080026101D
:1001B0002108A3020318E0280130A402031C26141E
:1001C0002208A402031C2614031026180314080096
:1001D0002730A2001030A1000121A7000330A200A7
:1001E000E830A1000121A800A2016430A100012192
:1001F000AA00A2010A30A1000121A9002308AB0036
:100200000800A501A50AD720031C0229D020250338
:1002100008008030762143308521203085213D3013
:100220008521A6142708242128082421203085218F
:100230002A08242129082421A6102B082421E4308F
:100240008521463085210800031DA6103038A618E8
:10025000203085210800B200C8307621B203362153
:10026000803E031885297F3985212F29B20A32085B
:100270008200FF30AC009721303086000614000069
:1002800006103230AC0097213030572130305721E2
:100290002030572101307621283076210830762110
:1002A00006307621033076210C3076210800860056
:1002B0000614000006100A30AC00972108008316CF
:1002C000F030860483120611861506140000060815
:1002D000AE0006100000061400000610AE1B6329D5
:1002E000861183160F30860583120800AF005F2148
:1002F0002F08F03986000614000006102F0EF03982
:1003000086000614000006100800AF005F212F08C9
:10031000F039860006150614000006102F0EF0397D
:100320008600061506140000061006110800FA30B3
:10033000AD00000000000000000000000000000010
:0A034000AD0B9929AC0B972900348E
:02400E00323F3F
:00000001FF
